:020000020000FC
:1000000085CEC0C10000000020C000008DC00000EF
:10001000000097C00000000000000000020304067A
:10002000080C10182030406080000406080C1018DE
:100030002030406080A0C0000003070F1F000D0D9E
:100040000403060D0503030202004FB662FD0CC057
:10005000552041F00994C52DC095089483FDC7959E
:10006000C4BD64604FBE1895C0916400089483FDC0
:10007000C795C4BD6B7FC0916400CF3F09F41DC01C
:1000800070FF19C082FD05C04FBEC098C198C298CC
:100090001895C098C198C29876FD0DC064FD0BC03C
:1000A000C9E0CA95F1F7C091B100C0FD939AC1FDB6
:1000B000949AC2FD959A4FBE189524BCCC27C06473
:1000C000C8BF6460F8CFC7CF70FFC5CF64FDC3CF92
:1000D000C09AC1CF70FFBFCF64FDBDCFC19ABBCF67
:1000E00070FFB9CF64FDB7CFC29AB5CF939870FFB8
:1000F000B2CF64FDB0CFC7E0CA95F1F7C09AABCFDD
:10010000949870FFA8CF64FDA6CFC7E0CA95F1F719
:10011000C19AA1CF959870FF9ECF64FD9CCFC7E098
:10012000CA95F1F7C29A97CF4FB6C9B7CF7EC9BF6C
:100130006E7FCCB5CE0DDDB5DF1DDBBDCABD4FBEBC
:1001400018953FB68F7EABB7A074A2118061A0E076
:10015000ABBFA9B7AE7FA9BF7894A0916800AA23CE
:1001600041F085FD2EC0A0916800AA95A09368007B
:1001700028C040E050E085FD14C0A0B396FDA095D6
:10018000A2FD4FEFA3E096FDA2E0A5BFAA27A064C1
:10019000AABF8D7FA0B396FDA095A2FD5FEF451786
:1001A00041F7A0E461FDA093680085FD03C0A0E4D1
:1001B000A0936800409396008160442311F0209240
:1001C000990085FD0EC0A0916900AA2331F0A0918D
:1001D0006900AA95A093690004C08061AA27A06461
:1001E000AABF80FF0AC0A09196004A2F61FF8E7FB0
:1001F00085FD01C000C0409361004091B4004430CF
:1002000009F004C0A0916100A0936300A091600078
:10021000A395A093600051F0F894A9B7A160A9BF7D
:1002200084FF02C0A0E4ABBF3FBE1895A09174004C
:10023000A395A093740042E050916800552329F0E3
:1002400085FF03C05A9550936800A0919600A13095
:1002500018F0209299000DC020929A002092A300DD
:10026000A0919900AF5FA093990018F0AFEFA09311
:100270009900B09061005091B400523049F465FF8C
:1002800091F0A2E3BA1678F0A0918600A0936100E5
:10029000533049F465FF39F0A2E3BA1620F0A0917B
:1002A000C000A0936100509162005B1521F010F036
:1002B0005A9501C05395509362004A95D1F65091DA
:1002C000A300539509F45A955093A300A091A4005C
:1002D000AA95A093A40009F04BC0A1E0A093A400AC
:1002E00048E0A091A500AA2381F145E0A091A500D6
:1002F0005A17F0F1A091A6005A1728F441E0A3E0A4
:10030000A093A40007C0A091A7005A1718F441E0D9
:100310004093A400D0909C00C0906300DC14A8F02F
:10032000A091B400A430D9F065FD0FC0C0929C002C
:10033000539521F0A091A500A093A300A1E0A09364
:10034000A400ACE3A093620013C0A0919C00A40F92
:1003500020F45FEF50939C0002C0A0939C00A091FA
:100360009C00AF3F29F4AFEFA0939A00A093A300A5
:10037000F894A9B7A160A9BF84FF02C0A0E4ABBFF5
:100380003FBE18953FB64CB55DB58F7EABB7A07438
:10039000A2118061A0E0ABBFA9B7AE7FA9BF7894DE
:1003A00081FD23C0A2E096FDA3E0A5BF8260A0B3BB
:1003B00096FDA095A2FF05C040936500509366008E
:1003C0001CC1A3E096FDA2E0A5BFAA27A064AABF16
:1003D0008D7F85FF01C004C140E0A0B396FDA095CC
:1003E000A2FDFEC040939600EDC0A3E096FDA2E002
:1003F000A5BF8D7F61FF71C0A2E096FDA3E0A5BF00
:10040000AA27A064AABF82604093910050939200F3
:10041000A0908F004A19B09090005B09BB24A22CD9
:100420004C38520518F42092950049C0A091D40090
:10043000AA2359F1483C520528F4A0E1BA2EAAE0BB
:10044000AA2E23C04836A1E05A0728F4A8E0BA2E05
:10045000AFE0AA2E1AC0403DA2E05A0728F4A4E05B
:10046000BA2EAEE1AA2E11C0403AA5E05A0728F4F0
:10047000A2E0BA2EACE3AA2E08C04839A8E05A0779
:1004800020F4A1E0BA2EA8E7AA2EC42EA0919300D2
:10049000CA1AD52EA0919400DA0ADD202AF4AFEF13
:1004A000C094D094CA1ADA0A20929500A8E0A2104B
:1004B000A0E0CA14DA0618F4A1E0A09395004093D6
:1004C000930050939400409191005091920040937A
:1004D0008F005093900042E075C0A09165004A1BC8
:1004E000A09166005A0B94FD60C093FD5EC092FD22
:1004F0005AC086FF03C0D52EC42E0CC05695479512
:1005000091FD51C05695479590FD4DC0D52EC42EF6
:10051000D694C79461FD19C0AC2DAC51AD2DA2404D
:1005200008F005C0DD2089F4AC2DA85C70F4A09122
:100530006700A395AA2311F0A0936700AA3008F4DE
:100540004FC02092960081604BC0A0916700AA2303
:1005500019F0AA95A0936700A22C5091BA0097FDBC
:1005600002C0A090C800AAEFAA0EA22DA21DCA1810
:10057000DA0A4FB74170442319F040E050E015C04B
:10058000AFEFCA16D20418F04FEF50E00EC0A091A2
:10059000AC00CA9E412D000C441F50E008F012C070
:1005A0004FEF50E00FC05695479594FF07C0552375
:1005B00009F04FEFA42FA6954A0F521D4F3F520549
:1005C00008F04FEF40939600816061FF09C0AFE1F2
:1005D000A095A923AB299A2F8F7DBB2009F48062B7
:1005E000A0E4A093680085FF03C0AAE0A093680080
:1005F00061FD03C085FD01C08F7E85FD03C0A0E2C3
:10060000A0936900F894A9B7A160A9BF84FF02C0B4
:10061000A0E4ABBF3FBE189511E00AC013E008C0CC
:100620001AE006C01EE104C014E602C018EC00C0C7
:1006300005E1BB27BA95F1F70A95D9F71A95C1F7E5
:1006400008952AE338E709C020E33CE806C02AE21F
:1006500034EB03C025E238EC00C0B091AD00BA9590
:1006600009F4089512E0BB279498BA95F1F7C19A5E
:10067000BA95F1F7C198BA95F1F7949ABA95F1F74E
:10068000123009F0C09A123009F4C29AB091AD004C
:10069000BA95F1F7123009F0C098123009F4C298F7
:1006A000B7E8BA95F1F71A95F1F6022FB22FBA957D
:1006B000F1F70A95D9F73A9581F694980895221B97
:1006C00039E0001F3A9509F40895221F211B18F400
:1006D000210F8894F6CF0894F4CF622C722CB0E0EE
:1006E0008894B395221F331FE0F737952795889498
:1006F000912E802E020B130B10F4192D082D10F4DF
:10070000889401C00894661C771CBA9571F7172D60
:10071000062D0895322D11232AF43A95009510954F
:10072000031B130BF894029F712C002D129F912C28
:10073000802C7894780C172D921C292DB4E06B2E08
:100740002695179507956A94D9F7332321F00095DC
:100750001095031B130B08950091B400043009F4A5
:1007600074C0B0919600B95198F0B72FB67081F46B
:1007700065FD2BC005E09090C600B92DBA9521F01B
:100780000AE0BA9509F002E1B0917B00B01BE0F0FD
:1007900065FF0AC0B0919E00B0939C00BFEFB0937C
:1007A000A300B1E0B093A400B0916100B0936300E6
:1007B00020927E0020927F00209280002092810073
:1007C000209282006F7D41C060629090C600B92D7A
:1007D000BA9579F4B0916200B095BB1FBB1F1B2F77
:1007E000B7950B2FB12FB170B3951B2FB02FBE7FD4
:1007F00025C0B92DBA95BA9581F4B0916200B09533
:10080000BB1FBB1FBB1F1B2FB7950B2FB12FB37087
:10081000B3951B2FB02FBC7F14C0B0916200B09570
:10082000BB1FBB1FBB1FBB1F1B2FB7950B2FB12FB0
:10083000B770B395B3951B2FB02FB87FB0540B2F63
:10084000120900937E0010937F00089510917B00A1
:10085000169500917A000795B0917E00B01B0B2F82
:10086000B0917F00B10B1B2F28F40038BFEF1B079E
:1008700040F009C00F37120508F405C00FE710E07B
:1008800002C000E81FEF00938300109384000895D6
:1008900000918300B09180000B0F10918400B09103
:1008A00081001B1F20E03091840033230AF42A9535
:1008B000B09182002B1F1AF4203F40F00AC02F3065
:1008C00008F407C00FEF1FEF2FE003C000E010E0B7
:1008D00020EF30916300B0919B003B1718F4323049
:1008E00030F009C0B0918400BB235AF004C0B0912D
:1008F0008400BB2332F40093800010938100209386
:10090000820008952091D70000918300000F10917C
:100910008400111FFFDE11232AF40038BFEF1B07EC
:1009200040F009C00F37120508F405C00FE710E0CA
:1009300002C000E81FEF002352F0B0916200B01B2C
:100940000B2F18F0013008F00AC001E008C0009534
:100950000F5FB09162000B0F08F001C00FEF009322
:10096000850008952091D8000091810010918200A7
:10097000D1DE11232AF40130BFEF1B0740F009C07C
:100980000F3F120508F405C00FEF10E002C001E0B0
:100990001FEF112352F0B0918500B01B0B2F18F000
:1009A000013008F00AC001E008C000950F5FB09167
:1009B00085000B0F08F001C00FEF0093630008954E
:1009C0000FEF71FD1EC0B091D300BB23D1F0B091E9
:1009D0007B00BB23B1F00FEF10917B0070DEF89429
:1009E000B091730072FDB5E00B9F112D002D78942E
:1009F000112309F00FEFB0919E000B1710F4009136
:100A00009E0000939D00089500917A0010917B0054
:100A100000541140B0919D0010F4BA9501C0B395F7
:100A200011F0B0939D000895F8D3B0E074FDB1E0EB
:100A3000B06CB7B9B6B1B068B064B6B9EDDDB0E0CE
:100A400074FDB1E0B06CB7B9B6B1B068B064B6B916
:100A5000B6B1B6FDFDCF04B115B1B6B1BF77B6B929
:100A600033D42DE62093A800222309F441C030E0BE
:100A70003093A900732E7694622E6694620E731ED4
:100A8000262D372D0217130778F08090A800BDE6B9
:100A9000B80DB093A8008090A900B0E0B81DB09345
:100AA000A900260D371DEECF8090A8009090A900D8
:100AB0001091A90016950091A80007951695079525
:100AC00023E0169507952A95E1F72091B5002A9520
:100AD00029F42092A8002092A9000AC02A9521F0AA
:100AE000800E911E2A95E1F78092A8009092A900AD
:100AF00008952091B500B6B1B6FDFBCF04B115B194
:100B0000B6B1BF77B6B9B091AA00B395B093AA00B9
:100B1000B83060F12092AA00B091D200BB2321F13D
:100B2000112329F0B091AB00BF3F61F009C0B09133
:100B3000AB000B1739F020F4BB2321F0BA9502C0AB
:100B4000B395E1F300919B00B093AB00BA3F50F432
:100B500000ECB93F38F400E8B83F20F400E4B73FB8
:100B600008F400E000939B007F7E08952130B1F0EF
:100B70000F3FB3E01B0790F4BDE6BB2379F0B091C3
:100B8000A8000B17B091A9001B0740F4B0919B007F
:100B9000BB2359F0BA95B0939B0007C0B0919B005E
:100BA000BF3F19F0B395B0939B0000919B00B091AB
:100BB0006300B01B10F400916300B0919C000B1710
:100BC00050F000919C00B0919C00BF3F21F0B0918B
:100BD0009C00B0939B00502E00936400B091AA003B
:100BE000B73009F47061089502E3F894B091D90028
:100BF0000B9F012D000C001F7894B0919B000B17E8
:100C000010F000919B000093610000936300502E50
:100C10000093640000939E00089520927A00B0EF44
:100C2000B0937B000895F8940CB51DB52091740025
:100C30007894309175006090760000937500109361
:100C40007600031B160971FD03C077FD80C028C024
:100C500070907700209377002709222319F00FEF77
:100C60001FEF0EC08090780090907900309378004C
:100C700060927900009175001091760008191909A9
:100C800020917A0030917B0036952795020F131F33
:100C900010F40FEF1FEF00937A0010937B002BC02E
:100CA00020917A0030917B003901B4E08B2EB2E0C4
:100CB0009B2E343040F08A949A94383020F072FDA4
:100CC00002C08A949A94769467948A94E1F72619DC
:100CD0003709992021F0169507959A94E1F7200F8E
:100CE000311F20937A0030937B0028F43FEF30933C
:100CF0007A0030937B00323008F4706871FF02C0D4
:100D0000B3E00DC0B091C40000917100023838F01A
:100D1000B395003A08F0B395B63008F0B5E09B2ED5
:100D2000B4E08B2E10917B0000917A0024E01695A0
:100D300007952A95E1F70819120928F0B02FB2504B
:100D4000B12FB20910F402E010E0980126C0209102
:100D50007A0030917B0039017694679466946694AA
:100D600066942619320906950695200F321D2093A8
:100D70007A0030937B00323008F07F7704E03695BC
:100D800027953695279526952695201B10F022301D
:100D900008F422E089019090C40060FDFECFE0904D
:100DA0008B00F0908C006160B9B7B061B9BF3801B9
:100DB00077FD41C07694679400938B0010938C006C
:100DC000B92DB330E1F0B0FD04C0060D171D93013D
:100DD00006C0000F111F0250120922E030E0B92DA9
:100DE000B33068F020938D0030938E00009387001D
:100DF000109388006092890070928A003AC0009334
:100E00008D0010938E0020938700309388006092AD
:100E1000890070928A0071FF0DC0BFE0B0938D0011
:100E200020928E00B093890020928A00B0938B00AC
:100E300020928C001EC0669400938B00B92DB330B5
:100E400091F0B0FD03C0060D262D03C0000F025027
:100E500022E0B92DB33038F020938D000093870045
:100E60006092890006C000938D00209387006092F5
:100E7000890000917C0002FD0350013031F495FDA2
:100E80000FC0B0B7B77FB0BF11C0023039F4B0B7F0
:100E9000B860B0BFB4E0B06CB7B908C095FDF1CF91
:100EA000B0B7B860B0BFB5E0B06CB7B90091A20000
:100EB000000F10F4BBE60B270093A20060FDFECFED
:100EC000B2E0B0936E006160B9B7B061B9BFB72F3F
:100ED000B670D1F020917A0030917B00369527953D
:100EE0003695279571FF02C0B0E43B0FF8940CB51E
:100EF0001DB5020F131F1BBD0ABD6160B0E1B8BF75
:100F0000B9B7B061B9BF78940895686020927D0048
:100F100020E066FD20E206C0686020927D0020E2AD
:100F200066FD20E001E011E077FD11C0B72FB6703B
:100F300009F0677F14E100917B00069509F40395A1
:100F40000F3008F00FE071FF02C004E114E160FD12
:100F50000FC0B0917D00BB2359F071FF06C0B09166
:100F60006E00BA95B0936E0011F4706251C0ABDFA1
:100F7000B0B73B2FB77FB0BFB8B1B0B733FDB860E3
:100F8000B0BFB0917D00B395B0937D00B8B177FD4F
:100F900006C0B1E071FDB3E0BA95F1F7B8B1B07237
:100FA000B21709F02AC071FF05C00395011708F0B8
:100FB0000A95CDCF63FD05C00395011708F0B2CFA8
:100FC000C6CF677FF8943CB56DB470907A00B0914D
:100FD0007B00770CBB1F08F4BFEF770CBB1F08F436
:100FE000BFEF370D6B1E6BBC3ABD6160B0E1B8BF9F
:100FF000B9B7B061B9BF789495CFB0916D00B130F9
:1010000008F490CF63FD8ECF0A9509F0A0CF7F7DC5
:1010100020918D0030918E00F894B0E1B8BF0CB5EE
:101020001DB5020F131F1BBD0ABDE0908700F09095
:1010300088006160B9B7B061B9BF7894B72FB67056
:1010400039F0B0916D0072FFB395B0936D0009C097
:1010500075FF07C066FD05C063FD03C0BF91BF916A
:10106000FCC4089500E063FF01C001E0F894109112
:101070007100B7E01B9F212D102D7894200F26952D
:101080001795269517952695179510937100183783
:1010900018F4B8E7B093710000917100B09172003C
:1010A0000B1720F06061C098C198C29860FDFECF18
:1010B000E0908900F0908A006160B9B7B061B9BF73
:1010C0000895B2E095FD0AC0F894B0937C0094981E
:1010D000939A62FF01C0C29A7894F4C0F894B093D6
:1010E0007C009498959A62FF01C0C09A7894EAC0F7
:1010F000B3E082FF24C095FD11C002E0F894B093E4
:101100007C00E0E8F0E00093B100C298959862FF9F
:1011100002C0C19A01C0949A7894D4C002E0F894B5
:10112000B0937C00E0E8F0E00093B100C0989398A1
:1011300062FF02C0C19A01C0949A7894C3C095FD21
:101140000BC0F894B0937C00EAE6F0E0C29862FF2E
:1011500001C0C19A7894B6C0F894B0937C00EAE6D6
:10116000F0E0C09862FF01C0C19A7894ABC0B4E0CF
:1011700095FD0AC0F894B0937C009398959A62FF0D
:1011800001C0C19A78949EC0F894B0937C00959861
:10119000939A62FF01C0C19A789494C0B5E082FF2F
:1011A00024C095FD11C001E0F894B0937C00E6E7FF
:1011B000F0E00093B100C198949862FF02C0C09A19
:1011C00001C0939A78947EC004E0F894B0937C00B8
:1011D000EAE8F0E00093B100C198949862FF02C081
:1011E000C29A01C0959A78946DC095FD0BC0F89491
:1011F000B0937C00E4E6F0E0C19862FF01C0C09AC1
:10120000789460C0F894B0937C00E0E7F0E0C19877
:1012100062FF01C0C29A789455C0B6E095FD0AC03D
:10122000F894B0937C009598949A62FF01C0C09A9C
:10123000789448C0F894B0937C009398949A62FF95
:1012400001C0C29A78943EC0B1E082FF24C095FDEF
:1012500011C004E0F894B0937C00EAE8F0E0009359
:10126000B100C098939862FF02C0C29A01C0959ADB
:10127000789428C001E0F894B0937C00E6E7F0E0B1
:101280000093B100C298959862FF02C0C09A01C055
:10129000939A789417C095FD0BC0F894B0937C0096
:1012A000E0E7F0E0C09862FF01C0C29A78940AC0FB
:1012B000F894B0937C00E4E6F0E0C29862FF01C0CD
:1012C000C09A78946F7E089523E630E0F901209269
:1012D000B100C098C198C2989398949895986B7FE4
:1012E0000895A2EBB0E007E00D9307E00D9301E055
:1012F0000D9304E00D930FEF0D930D9309E00D9303
:1013000002E00D9301E00D9301E00D93AEEBB0E030
:1013100001E00D9300E00D9304EB0D930FEF0D939F
:101320000D930D9303E00D930FEF0D9301E00D93DB
:101330000FEF0D9305E20D9300ED0D9308E70D936C
:1013400008EC0D9304E00D930FEF0D9301E00D9366
:1013500000E00D930AE70D930AE00D9300E00D9372
:1013600001E00D9300E00D930FEF0D9300E00D935E
:1013700008952091B9008B7F233009F48460B091E7
:10138000BA009F7DB1FD90629F7BB091BB00B1FD23
:101390009064223011F0886001C0877F08950A951B
:1013A000E00FF21DB4910895ECE1F0E00091B2007D
:1013B000F6DFB093D700ECE1F0E00091B300EFDF8F
:1013C000B093D800EAE2F0E00091B800E8DFB09313
:1013D000D9000091D100002319F42092A50013C078
:1013E000013108F001E1B02FB00FB00FB093A500AC
:1013F0001B2FB10FB10FB00FB093A600B10FB00FFC
:10140000B00FB093A7000091B800023008F402E0DA
:1014100000937300B091CE000FEFB23009F400EAF0
:10142000B33009F402E800937200E8E3F0E00091C1
:10143000D500B5DFB093A000089508952091C800AD
:101440003091C900B091BA00B33009F43E5097FF13
:1014500002C020E03FEFB32FB21B6B2EB25810F446
:10146000B2E86B2E00E00395609EB12DBD57D8F316
:101470000093AC0008959068E1DFD4D8D3D820E081
:1014800030E0B0E16B2ECAD8B09196002B0F321D20
:101490006A94C9F7B4E036952795BA95E1F7822E9C
:1014A0009F77CCDF0895F894E3E0F0E0B9E0B7BFB0
:1014B000B491B078C1F3F894A895B1B5B861B1BD55
:1014C000B0E0B1BDB4E0BEBFBFE5BDBFFDDEB0E082
:1014D000B8BBB7E1B7BBB0E0B5BBB0E0B4BBB0E000
:1014E000B2BBB8E3B1BB2224A0E0B0E02D92AA3198
:1014F000E9F7A0E6B0E00FEF2D920A95E9F7B1E029
:10150000B093A200EEDEEAD2B0E0B06CB7B9B6B1EB
:10151000B460B068B6B90091CA000093AD00B1E004
:10152000B0936A00F89482D88CD87CD88DD87AD8B9
:101530008ED878D862D37AD879D876D8F8940AEF4A
:101540001AEFA0B396FDA095A2FF1FC01A95C9F788
:101550000A95B1F7E0E0FCE1B591B43E39F4B591FC
:10156000B03E21F4B591BF3F09F40CC0E0E0F39523
:10157000F395B591B83F49F4B591B43931F4B591CB
:10158000BA3A19F4EE27F6950994F3DE0DDF55DF2C
:1015900055DF0091CA000093AD0096DEB2E0B3BF04
:1015A000B2E0BEBDB2E0B5BDB1E5B8BFB9BFB0B73E
:1015B0000B2FB77FB0BFB8B1B0B703FDB860B0BFF5
:1015C0002BD8789431DA20927000B3E096FDB2E027
:1015D000B5BFB0E4BBBFBB27B064BABF8D7F26D810
:1015E000626033E02CE0B0919500BB2321F42CE045
:1015F0003A9509F4A3CF16D880FFA0CF8E7FB09183
:101600009600B23078F3B92FBF7100919800009323
:101610009700B0939800B01729F72A9521F76D7FAE
:10162000B3E096FDB2E0B5BFBB27B064BABF8D7F13
:10163000B091D400BB2321F48062B92FB0709B2FEE
:101640008F7B20926700F0D785FF05C0B0916700BF
:10165000BA3008F08064E2D702E085FF01C000E004
:10166000B0919600B017B8F3F894EBD7EAD7E9D762
:101670007894DCD720928600D1D7B091BE00B130EB
:1016800008F478C0B0916A00B13008F473C085FDE9
:1016900018C0B0919600BF3F08F46CC0F894DAD738
:1016A0007894C2D7B0919600B130C0F7F894C9D7FA
:1016B000B7D7C7D77894B8D7B0919600BF3FB0F3EB
:1016C000CEC2B8E09B2E9068F894B8DE7894ACD780
:1016D000F8949F77B3DE80909600B0919600BF3764
:1016E000789408F44FC098D7F894B4D778949A9423
:1016F00051F7C1DEB82DB550B093C90097D7F89413
:1017000081D27894BAE09B2E9068F89497DE789412
:101710008BD7F8949F7792DE80909600B0919600D8
:10172000BF37789478F778D7F8948BD779D789D75B
:1017300078949A9449F79FDEB82DBB5FB093C800A8
:101740000B2F1091C900125810F0100B20F4B2E8C2
:101750000B0F0093C9006AD7F894EDD162D2789448
:1017600063D7F8946BDE7894B0919600BF3F08F48D
:101770008ECF75C200919600B09186000B1710F0C5
:101780000093860051D701E0B091BA00B35009F43C
:1017900005E0B0919600B01708F06ECFF8945AD7D4
:1017A00059D758D7789442D720926A0020926B007C
:1017B00020926C00B0916B00B395B0936B00BF3F6B
:1017C00071F5B0916C00B395B0936C00B091CC0002
:1017D00009E1BA9559F002E3BA9541F00DE7BA95DF
:1017E00029F00AEFBA9511F020926C00B0916C00CC
:1017F000B017A8F069DD10D7B0916C00BA95B0931E
:101800006C0020926B00B091CB00B093AD00F894C7
:1018100021D77894B091CA00B093AD0005D700D716
:10182000B0916800BB2319F485FF01C087CE01E0A9
:1018300085FD01C006E0B0919600B01708F4BACF5C
:10184000F3D6B0916800BB2309F478CEF8943CDD60
:10185000209261002092620020926300522C20921C
:1018600064002092A1007894B091B700BB0FB093B0
:101870009F0020927E0020927F0020928000209284
:101880008100209282002092AA0060E070E0209205
:101890007100B8E0B093AA007061BED6B0E074FDEC
:1018A000B1E0B06CB7B9B6B1B068B064B6B9B6B1B2
:1018B000B6FDFDCF04B115B1B6B1BF77B6B91123EE
:1018C00009F00FEF0093AB0014D9B8E0B093AA0071
:1018D00070614FDDF894BFEFB0939B0085D9B09154
:1018E0006100B0939B00B0939C00B0939D007894EE
:1018F000B1E0B0936100B09363005B2EB0936400DD
:10190000B093A400B0919A00B093A300B091BA0034
:10191000B33019F49F7D87FD9062716072602092F0
:101920006D007BDC91DC79D97ED977D97CD975D9EA
:10193000F3DA12D797DBC5DB76D9E7DA65FD86D710
:1019400077FF3ED877FD60D88DDBD2DB6CD9E4DA47
:1019500065FD9ED787DB0BDC66D9D7DA65FDD2D76C
:1019600081DB1CDC60D9D8DA65FDFCD77BDB55DC7C
:101970005AD9CBDAB0E074FDB1E0B06CB7B9B6B10A
:10198000B068B064B6B96EDB5FDC4DD9B2D871FF18
:101990001EC0B0919E00B0939B00B0939C00B0918C
:1019A0009A00B093A300B1E0B093A40018E12CE03A
:1019B000B0916D00B11728F07D7F746020936F00A7
:1019C00006C0B0919600B13008F0B2CF50C072FF9F
:1019D00015C066FD13C0B0916F00BA9519F47B7FF6
:1019E0007860A6CFB0936F00B0919600B13008F048
:1019F0009FCFB091BA00B33009F039C02092700087
:101A0000B0919900B13058F0B0919E00B0939C0015
:101A1000B0919A00B093A300B1E0B093A400B0914C
:101A200099000AEF1091D600112309F003E0B017D6
:101A300008F01DC085FF04C0B0916800BB23B9F059
:101A400000EF66FF05C0B0919E00B0939B0000E2DE
:101A5000B0917B00B01708F46BCFB0917000B395D4
:101A6000B0937000B0919600BB2309F002C02092A1
:101A70007000F89429DC8090B900B2E0B093B9000E
:101A800078DC8092B900209261002092620020925E
:101A90006300522C2092640020929F0060E070E06E
:101AA0007894C2D511DC0091D600002319F0C09AB9
:101AB000C19AC29AB0E0B06CB7B9B6B1B460B068C0
:101AC000B6B985FF05C0B0916800BB2309F436CDD7
:101AD000B091BF00B13008F0BECD68CEEDE0F0E0CF
:101AE00023D0053A09F01BC0EEE0F0E01DD00A3526
:101AF00009F015C03AE0A2EBB0E0E3E0F0E014D06A
:101B00000D9331963A95D9F739E1AEEBB0E0EFE0BD
:101B1000F0E00AD00D9331963A95D9F702C0E1DB97
:101B20000AD0E8E2F0E00895E199FECFEEBBFFBBFA
:101B3000E09A0DB308951ED03AE0A2EBB0E0E3E0E6
:101B4000F0E00D910FD031963A95D9F739E1AEEB2F
:101B5000B0E0EFE0F0E00D9105D031963A95D9F77D
:101B600012D00895E199FECF0DBBEEBBFFBBE29A08
:101B7000E19A0895EDE0F0E00FEFF4DFEEE0F0E041
:101B80000FEFF0DF0895EDE0F0E005EAEBDFEEE0C7
:101B9000F0E00AE5E7DF08953091AE000091AF0074
:101BA000313011F40093B200323011F40093B300DD
:101BB000333011F40093B400343011F40093C600B4
:101BC000353011F40093B500363011F40093B800AD
:101BD000373011F40093C400383011F40093B90089
:101BE000393011F40093CE003A3011F40093BA006A
:101BF0003B3011F40093BB00089525E017D52A95DA
:101C0000E9F708951ED520D522D524D509D519D5B3
:101C10001BD51DD51FD504D514D516D518D51AD565
:101C2000089518D514D510D50CD5FAD413D50FD5E1
:101C30000BD507D5F5D40ED50AD506D502D508950E
:101C40008090AE009090AF00FCD4FBD4FAD4E8D4DE
:101C50008A94D1F7FFD4E4D49A94E1F70895F894E4
:101C6000D1DF7894CADFC9DFB1E0B093AE00B1E054
:101C7000B093AF002092B000F894E2DF7894B5E022
:101C80006B2E70909600D2D4B09196007B16C9F757
:101C9000B13018F0BF3F40F107C07EDFF8944BDF52
:101CA000B1DFB8E0B1BDA9DF6A9459F7B091B000D7
:101CB000B395B093B000B33008F4DECF9EDFB0919F
:101CC000AF00B395B093AF00F894B091AE00BA9561
:101CD000EEE3F0E0EB0FF21D049178940395B091E0
:101CE000AF00B01708F4C6CF88DF87DFB091AE0031
:101CF000B395B093AE00B091AE00BC3008F4B7CF4E
:0E1D0000F0DAF89418DFB8E0B1BD77DFCCCB95
:00000001FF
